:020000040800F2
:1000000070100020990100087B1200083D070008CD
:100010007912000883050008512100080000000043
:10002000000000000000000000000000AD15000806
:100030008505000800000000A5140008E915000867
:10004000B3010008B3010008B3010008B3010008C0
:10005000B3010008B3010008B3010008B3010008B0
:10006000B3010008B3010008B3010008B3010008A0
:10007000B3010008B3010008B3010008B301000890
:10008000B3010008B3010008B3010008B301000880
:10009000B3010008B3010008B3010008B301000870
:1000A000B3010008BD160008B3010008B301000841
:1000B000B3010008F1180008B3010008B3010008FB
:1000C000B3010008B3010008B3010008B301000840
:1000D000B3010008B3010008B30100083D1A00088D
:1000E000B3010008B3010008B301000800F002F8F2
:1000F00000F042F80AA090E8000C82448344AAF180
:100100000107DA4501D100F037F8AFF2090EBAE87D
:100110000F0013F0010F18BFFB1A43F0010318473B
:100120001860000038600000103A24BF78C878C119
:10013000FAD8520724BF30C830C144BF04680C60ED
:10014000704700000023002400250026103A28BF35
:1001500078C1FBD8520728BF30C148BF0B60704739
:10016000642900F07780732900F0C981002070476E
:100170001FB51FBD10B510BD00F0CEF91146FFF739
:10018000F7FF03F05BFC00F0ECF903B4FFF7F2FFBC
:1001900003BC00F0EFF90000094880470948004718
:1001A000FEE7FEE7FEE7FEE7FEE7FEE7FEE7FEE727
:1001B000FEE7FEE704480549054A064B7047000084
:1001C000B9160008ED00000870050020701000202E
:1001D00070070020700700200FB41CB5074B06AA5B
:1001E0007B4469460090059800F05FF9002069465D
:1001F00000F06EF91CBC5DF814FB0000ED0200007D
:1002000070B50C460546012A05D02878800600D531
:10021000EA69002302E0012305E05B1C934202D25D
:10022000E05C0028F9D1A869E618C01AA861286A1C
:10023000184428622846AFF3008004E0D5E9012184
:1002400014F8010B9047B442F8D32846AFF300806E
:1002500070BD00002DE9F0410646002410687529A4
:10026000314616A510D0AFF30080002802DA4042D4
:1002700013A507E031688A0701D512A502E04907F6
:1002800004D511A5012401E0AFF3008000210A226A
:1002900006F1240709E0B0FBF2FCB0FBF2F302FB2D
:1002A0001C00303078541846491C0028F3D12346EE
:1002B0002A463046BDE8F04100F099B80000000041
:1002C0002D0000002B000000200000002DE9F0416F
:1002D0000F460546002028622846E968884770B323
:1002E000252805D0D5E901219047286A401CF2E76E
:1002F000E9682846002688476C2804460AD0682CFE
:1003000008D04C2C35D06A2C31D0742C31D07A2CBA
:100310002FD016E0E968064628468847B0420446D2
:1003200008D16C2E23D04FF480662846E9688847B0
:10033000044606E06C2E03D04FF4807601E01EE008
:100340004026E4B1A4F14100192802D8203446F433
:1003500000663A46214628462E60FFF701FF60B14D
:10036000012808D0FF1D27F007070837B4E78026CB
:10037000DBE70026D9E73F1DAEE72046B2E7286A53
:10038000BDE8F0814FF0000200B513469446964652
:10039000203922BFA0E80C50A0E80C50B1F1200198
:1003A000BFF4F7AF090728BFA0E80C5048BF0CC046
:1003B0005DF804EB890028BF40F8042B08BF7047A4
:1003C00048BF20F8022B11F0804F18BF00F8012B16
:1003D000704770477047704710B500F095F8006897
:1003E00010BD10B5044600F08FF8046010BD2DE973
:1003F000F0470D4699469246044600F124080168EC
:10040000880604D5E06921F01001216000E0012098
:10041000A84201DD471B00E00027A1697A1902EB21
:100420000900081AA0612078C00602D42046AFF364
:100430000080002608E0D4E901211AF80600904760
:10044000206A401C761C20624E45F4DB2078C006F2
:100450000AD52046AFF3008006E0D4E90121302020
:100460009047206A401C2062381EA7F10107F4DC87
:1004700007E0D4E9012118F805009047206A401CE4
:100480002062281EA5F10105F3DC2046AFF30080B1
:100490002078000602D50220BDE8F0870120FBE7A6
:1004A00001694A1C02610878704700B58FB0CDE938
:1004B00001310021059105497944CDE90310114628
:1004C0006846FFF703FF0FB000BD0000E5FFFFFF28
:1004D0000A6802F8010B0A60704710B5436913B14E
:1004E000AFF3008001E0FFF78BFE012010BD127812
:1004F00000F124010A7000224A700122EDE7116820
:100500004FF0FF32E9E70000004870470C0500207B
:10051000004870470C0500207546FFF7F9FFAE460E
:1005200005006946534620F00700854618B020B5FF
:10053000FFF740FEBDE820404FF000064FF00007F7
:100540004FF000084FF0000B21F00701AC46ACE87B
:10055000C009ACE8C009ACE8C009ACE8C0098D46E8
:10056000704710B50446AFF300802046BDE8104048
:10057000FFF70BBE01491820ABBEFEE726000200C4
:100580007047FEE7704772B6FEE700000422064B94
:100590000649002803D01A61886A086202E05A619D
:1005A000486A086201F014B8000801408000002089
:1005B00000B5012000F0F2FF0246022000F0EEFF3D
:1005C0001044801CC2B2642002F0B0FE002000F093
:1005D000E5FF0346032000F0E1FF0344042000F0A0
:1005E000DDFF1844C01CC0B202B9032218B10021BB
:1005F000FF2808D000E001210023194300D0072282
:1006000042EA002000BD0123F7E7000002488168AC
:1006100002781144816070471001002010B507482E
:10062000016841F010010160032000F061F80F2023
:1006300000F006F800F026F8002010BD002002406F
:1006400070B504460D4D4FF47A712878B1FBF0F087
:100650000B490968B1FBF0F000F05CF808B101202B
:1006600070BD102C07D200222146501E00F020F849
:100670006C60002070BD012070BD000010010020E2
:100680001C01002008B50948816941F00101816120
:10069000816901F001010091C16941F08051C1619E
:1006A000C06900F08050009008BD000000100240BA
:1006B000F0B40D460D4B1B68C3F30223C3F10704CE
:1006C000042C00D90424191D072901D2002300E0BD
:1006D000DB1E012606FA04F1491E294099409E407E
:1006E000761E16403143F0BC01F046BE0CED00E032
:1006F00000F00701054A10684FF6FF03184040EA72
:100700000120034908431060704700000CED00E031
:100710000000FA0510B5401EB0F1807F01D3012022
:1007200010BD4FF0E02460610F21601701F024FE3E
:100730000020A06107202061002010BDFEE700001E
:1007400030B5114B80251D60962002F0EFFD402250
:100750001A60962002F0EAFD4FF4167002F0E6FDF2
:10076000094C241D2260962002F0E0FD1A609620BC
:1007700002F0DCFD2560962002F0D8FD2260BDE885
:100780003040962002F0D2BD100C014000B509485F
:1007900080220260962002F0C9FD064B40201B1FFC
:1007A0001860962002F0C2FD1A6096205DF804EBF6
:1007B00002F0BCBD140C0140F0B503460022134EFC
:1007C0008025371D4024180601D5356000E03D60C6
:1007D000962002F0ABFD3460962002F0A7FD3C604D
:1007E0005806030E521CD2B2082AECD3962002F00F
:1007F0009DFD3460962002F099FD04480838006899
:1008000040F3C010401C3C603D60F0BD100C014046
:1008100070B50023144905200860142002F086FDFD
:100820000022114C4FF49675343CA06840F4A000AF
:10083000A060142002F07AFDE06C80B2984200DDE6
:100840000346521CAA42F0DBA3F11B00002800DA89
:10085000002004F038FC0022044B04F043FABDE809
:10086000704004F0D3BB0000342801400000F83F82
:100870000D49CA68D207FCD1CA6893064FF020021E
:1008800000D5CA600B6943F002030B614861086937
:1008900040F040000861C8688006FCD5CA6008695D
:1008A00020F002000861704700200240F0B5114CB2
:1008B000E368DB07FCD1E3684FF020069B0600D518
:1008C000E660236943F00103236100230AE0C718AF
:1008D000C55C7F7805EB0725CD52E568AD06FCD5F4
:1008E000E6609B1C9342F2D3206920F00100206156
:1008F000F0BD00000020024070B54FF400546200CB
:10090000104953004A2803DD0C614A614B6170BDF8
:10091000312803DD0B614C614A6170BD6FF009063F
:10092000B04203DD0A614C614B6170BD0025B042ED
:1009300001DA012000E000200543F6D04A614B6156
:100940004C6170BD000C014010B500220C4B9B683F
:10095000C3F300030B4CA468C4F30004234302D088
:100960000122104610BD096829B1436823F47023A1
:100970000B434360F5E7416821F470214160F0E7E3
:10098000002401400028014010B500228368C3F311
:100990000003002B02D00122104610BD43684C68B2
:1009A00023F48073234343608368096823F400635E
:1009B0000B438360F0E7000070B500234A68846849
:1009C000C4F30004002C02D00123184670BD3AB1D4
:1009D0008C682243446824F468442243426003E064
:1009E000426822F468424260CC680A688568224303
:1009F0000C69064E35402C43224382604968C26A26
:100A000022F470020A43C262DFE70000FDFEF1FF3C
:100A100010B54FF4407494FAA4F401F44073B4FA9E
:100A200084F4E34000EB8300C36A01F01F011F243C
:100A30008C4002F01F02A3438A401343C36210BDDF
:100A400070B54FF0007494FAA4F401F00073B4FA96
:100A500084F4E34000EB8300C4684FF0F87393FA2A
:100A6000A3F501F0F871B5FA85F521FA05F5072629
:100A7000AE4093FAA3F3B3FA83F3D940B4438A4068
:100A80001443C46070BD000008B50449CA6902433C
:100A9000CA61C9690140009108BD00000010024010
:100AA00008B504498A6902438A6189690140009155
:100AB00008BD0000001002402DE9F0410A68C2F3B1
:100AC0000F2595FAA5F2B2FA82F26BE0012393406A
:100AD0002B4266D0082A03D240F20113934006E06D
:100AE000A2F108034FF001149C4044F080634C686D
:100AF000082C0BD10C69C6681F0A97FAA7F7B7FA3A
:100B000087F726EA1326BC402643C6604F6800EBF1
:100B1000136493FAA3FCBCFA8CFC4FEA8C084FF0E8
:100B20000F0C26680CFA08FC26EA0C0693FAA3FCC4
:100B3000BCFA8CFC4FEA8C0C07FA0CF73E4326609B
:100B40004F68012F01D0092F2BD18F6893FAA3FC96
:100B5000BCFA8CFC4FEA8C084FF0030C0CFA08FC32
:100B600026EA0C0693FAA3FCBCFA8CFC4FEA8C0C28
:100B700007FA0CF73E432660CF6893FAA3FCBCFA51
:100B80008CFC4FEA8C084FF0040C0CFA08FC93FA2A
:100B9000A3F3B3FA83F39B0026EA0C069F403E437F
:100BA0002660521C35FA02F390D10020BDE8F08196
:100BB0008068090A81430804000C01D000207047B6
:100BC0000120704700B5034600F098FC186000F063
:100BD0006BFC586000F076FC9860586800F080FC70
:100BE000D86000BD01490860704700001C0100206A
:100BF000F0B50268154D164B164C4FF08046A842D2
:100C000005D0B04203D0984201D0A04203D14F6832
:100C100022F070023A43A84205D0B04203D0984275
:100C200001D0A04203D1CB6822F440721A43026083
:100C30008A68C2620A888262A84201D10969016396
:100C4000416941F0010141610020F0BD002C0140EB
:100C500000040040000800400346012001290BD099
:100C600010290DD0B1F5807F0ED0B1F5805F0FD186
:100C70001146184600F0C4BB1146184600F018BBD8
:100C80001146184600F04ABB1146184600F080BBDA
:100C9000704700002DE9FF4104460E46012700255C
:100CA000E068C0F3403000285DD1F1687068E26808
:100CB0000843316941F20C639A4311430843E060F1
:100CC000B068216921F44051014321617069616973
:100CD00021F44071014361616846FFF773FF2448C6
:100CE000844201D1039D08E02248844201D1029D43
:100CF00003E02148844200D1029DA5B3306890B33F
:100D0000002705EBC50101EB05118000B1FBF0F3F5
:100D10006422B3FBF2F36FF018067343B1FBF0F5F6
:100D2000B1FBF0F605EB8305322303EB0515B5FBAC
:100D3000F2F5B6FBF2F605F0F00505EB0615B1FB92
:100D4000F0F6B1FBF0F0B0FBF2F06FF018014843A1
:100D500006EB800003EB0010B0FBF2F000F00F0098
:100D6000284480B2A06004B03846BDE8F08100009D
:100D700000380140004400400048004008B54FF0F2
:100D8000E0210A690092421C05D0401C03E00A6978
:100D9000D20300D5401E0028F9D108BD70B58EB031
:100DA00000240C940D940B94142106A8FFF7EAFA82
:100DB000142101A8FFF7E6FA4FF400752846FFF763
:100DC0006FFE0420FFF76CFEA81C0190029401A99D
:100DD0001948FFF771FE01F0B7FA0122114600F041
:100DE0004DFA0146122001F0B7FA122001F08EFAF6
:100DF0000C940D94114E0CA93046FFF7C5FD0B94D1
:100E00000BA93046FFF7A0FDA802069007940894AE
:100E100009940A9406A93046FFF7CEFD084C2946EE
:100E200022463046FFF7F4FD002221463046FFF708
:100E300007FE0EB070BD0000000801400024014014
:100E40000100300230B58DB000240B940C941421B5
:100E500006A8FFF797FA142101A8FFF793FA4FF4B9
:100E60008060FFF71DFE0420FFF71AFE42F22110FA
:100E70000190029401A91848FFF71EFE01F064FAE0
:100E80000022114600F0FAF90146122001F064FA3E
:100E9000122001F03BFA0B940C94104D0BA928463C
:100EA000FFF772FD4FF460210691079408940994AE
:100EB0000A9406A92846FFF77FFD4FF000742246EA
:100EC00021142846FFF7A4FD002221462846FFF7FB
:100ED000B7FD0DB030BD0000000801400028014002
:100EE0002DE9F04F85B014216846FFF74BFA10202A
:100EF000FFF7D6FD2020FFF7D3FD0420FFF7D0FD3C
:100F00000820FFF7CDFD234C234F4FF400407861BC
:100F1000DFF888A0DFF8888048F2C400C8F8140021
:100F2000DFF880B0DFF880904FF20810C9F81400A5
:100F30001E4800900420019069463846FFF7BCFD2A
:100F40000094012401940225029500260396694627
:100F50003846FFF7B1FDCDF800A001940295039645
:100F600069464046FFF7A8FD41F2100000900820B6
:100F70000190049469464046FFF79EFDCDF800B00D
:100F800001940295039669464846FFF795FD05B022
:100F9000BDE8F08F8000800400100140C4C48004CC
:100FA00000080140F908F104000C01402000200471
:100FB00009498020086008481038026822F0704211
:100FC00042F0E042026040220A60016821F0706154
:100FD00041F0E06101607047100C01400B494CF694
:100FE000CC40086045F2555008600520486040F646
:100FF000FF708860C868800706D000200128F9D1FA
:101000004AF6AA20086070470120F7E70030004048
:1010100010B586B0142101A8FFF7B4F94FF40060B1
:10102000FFF73EFD01F090F90222114600F026F98B
:101030000146192001F090F9192001F078F949F6DC
:101040003F40ADF80400002002901321039104906A
:1010500005900C4C01A92046FFF7CAFD206840F01E
:1010600080002060A06844F207018843A0606068A7
:1010700020F070006060A06820F08000A06006B0E2
:1010800010BD0000002C01402DE9F04192B0142168
:101090000DA8FFF777F9202105A8FFF773F91421B0
:1010A0006846FFF76FF90120FFF7EEFC0927ADF85E
:1010B000347000260E964FF496600F901096BD0780
:1010C0000DA92846FFF794FD286840F080002860AD
:1010D000A86844F207018843A860A9141C488479D1
:1010E00004F1804418342068DFF86480082208F195
:1010F000070898F806309A40104320606020059059
:10110000069607960896099605AA2846FFF7A4FDB5
:10111000216898F806200420904081432160686887
:1011200020F070006860A86820F08000A8600420AB
:10113000FFF7B6FC40F608000090019702200290ED
:10114000039669460348FFF7B7FC12B0BDE8F0818B
:101150000A5E00080008014010B586B0142101A8FD
:10116000FFF710F90220FFF78FFC01F0EDF80022E5
:10117000114600F083F801461D2001F0EDF81D2016
:1011800001F0D5F80020ADF804000290E0210391B1
:1011900004900C4C01A92046FFF72AFD206820F09E
:1011A00080002060A06844F207018843A060606866
:1011B00020F070006060A06820F08000A06006B0A1
:1011C00010BD00000004004030B58DB01C2106A801
:1011D000FFF7D8F8142101A8FFF7D4F84FF48020C6
:1011E000FFF752FC0820FFF75BFC1F480190092025
:1011F000029003200390002404941C4D01A928466A
:10120000FFF75AFC1A4901910421029101A92846CD
:10121000FFF752FC01F098F80122114600F02EF879
:101220000146272001F098F8272001F080F84FF4BC
:10123000165006900794089409940C200A900B9479
:101240000C940C4C06A92046FFF724FD206920F4DD
:1012500090402061606920F02A006061E06840F4FD
:101260000050E0600DB030BD04000404000C0140EB
:101270000800080400480040FEE7FEE730B500F033
:101280000703C3F10704042C00D90424181D072800
:1012900001D2002300E0DB1E012505FA04F0401E08
:1012A000084098409D406D1E1540284330BD000009
:1012B00030B5026A22F001020262026A4368846960
:1012C00024F003040D6824F070042C430D6922F00F
:1012D00002022A434D6822F001022A430E4DA84221
:1012E00012D14D6922F0080242EA85028D6822F08F
:1012F000040242EA85028D6923F480732B43CD6991
:1013000023F4007343EA450343608461C968416381
:101310000262002030BD0000002C014030B5026A9E
:1013200022F010020262026A4368846924F4407465
:101330000D6824F4E04444EA05240D6922F02002FB
:1013400042EA05124D6822F0100242EA05120F4DE2
:10135000A84213D14D6922F0800242EA85128D68BD
:1013600022F0400242EA85128D6923F4806343EA49
:101370008503CD6923F4006343EAC50343608461B8
:10138000C96881630262002030BD0000002C01406A
:1013900030B5026A22F480720262026A4368C4694C
:1013A00024F003040D6824F070042C430D6922F42A
:1013B000007242EA05224D6822F4807242EA052258
:1013C0000E4DA84213D14D6922F4006242EA8522F3
:1013D0008D6822F4806242EA85228D6923F480536D
:1013E00043EA0513CD6923F4005343EA45134360F0
:1013F000C461C968C1630262002030BD002C014095
:1014000030B5026A22F480520262046A4268C369FB
:1014100023F440730D6823F4E04343EA05230D6988
:1014200024F4005444EA05344D6824F4805444EA1A
:101430000534074DA84204D18D6922F4804242EA66
:1014400085124260C361C96801640462002030BD36
:10145000002C0140104911484A6C0260104B501C8E
:10146000B3FBF0F040094FF47A7390FBF3F3083BC1
:1014700081F82D3001F1800318654001722390FB43
:10148000F3F020F01F0008654923B0FBF3F0486536
:10149000D008886570470000000000202C04004040
:1014A00000B4C404704700000449496801F0F00129
:1014B000034A0909515CC84070470000001002400F
:1014C000185E00080449496801F4E061034A02EB30
:1014D00011210978C840704700100240285E0008BA
:1014E0000449496801F46051034A02EBD1210978AB
:1014F000C840704700100240285E00080648406857
:1015000000F00C010548002905D0042903D0082962
:1015100001D100F005B870470010024000127A00B7
:101520000C4A506800F480300B49002809D0B0F50F
:10153000803F06D15068C0F34040401C4900B1FBD9
:10154000F0F1506800F47010022202EB9040484322
:10155000704700000010024000093D000449C978AE
:10156000494200EBC1200349084490F8000C704741
:101570000000002000F001080249084490F800042F
:101580007047000000D0010800F10060006870475B
:10159000014800787047000000DC01080249084457
:1015A00090F8E8077047000000F0FF1F7047000048
:1015B00000B5034605490A681206FCD50A2001F069
:1015C000B5FE0248001D036000BD00000048004059
:1015D00010B5044C206A03F099F9206ABDE8104068
:1015E00003F06CB980000020FFF710B810B52F4849
:1015F000016821F0070141F002010160016801F07A
:1016000007010229FAD12A4C206840F4803020607A
:101610002068C0F340400028FAD0606A40F0010022
:101620006062606AC0F340000028FAD0206840F48D
:1016300000202060606820F47C1040F4041060609A
:10164000206840F0807020602068C0F3406000286F
:10165000FAD0606820F0F0006060606820F4E0601C
:1016600040F480606060606820F460506060606892
:1016700020F0030040F002006060606800F00C00A1
:101680000828FAD10B48FFF7ADFA0F20FEF7D8FF74
:1016900008B1FEF778FF606820F4404040F48040D5
:1016A0006060606820F48000606010BD002002402F
:1016B0000010024000B4C404704700002DE9F05F40
:1016C00086480169C1F30001002902D06FF00101D1
:1016D0000161834DE86B401CE863287E00287DD1C2
:1016E0000024804E804606F1840956F8240004F058
:1016F00081F9AA7F214601F0C7FF04F03FF949F8BC
:10170000240046F82480641CE4B2202CEDD3FF2092
:1017100028762879401CC0B22871322803D985F870
:10172000078085F804806879401CC0B26871082879
:1017300002D16D4900034861C5F86880C5F864802E
:10174000674F8037C7F854800024DFF8A0B159F8FC
:10175000240004F04FF98246014604F077F9796DD0
:1017600003F0E2FF786550465BF8241004F06EF950
:101770000646686E04F03EF9314603F0D5FF04F0EA
:10178000FDF8686657495046843951F8241004F032
:101790005DF90646A86E04F02DF9314603F0C4FF4A
:1017A00004F0ECF8A866641CE4B2202CCFD36FF0F0
:1017B0000401786D04F0EBFA03F08AFF02F0F6FF03
:1017C00003F0A2F904467865686D04F02BF9014630
:1017D000204604F011F804F0EDF800E02CE0A864D5
:1017E0006A6E6A67A96EA967EC7E34B108203B680F
:1017F0009A4204DD03443B6003E00120F7E71B1A33
:101800003B60EB6F994202DD1844E86701E0181A6B
:10181000E867E87D18B185F817803A60E9673868AD
:10182000101A6867EA6F891AA96754B17861B961BB
:101830007869E866B8692867012085F82500BDE861
:10184000F09F95F82810012904D0022912D003290D
:1018500020D02EE004F0CEF801F072FD04F08EF8F6
:101860007861A86F04F0C6F801F0DCFD04F086F89A
:10187000B8611EE004F0BEF801F088FD04F07EF8C7
:101880007861A86F04F0B6F801F0F2FD04F076F884
:10189000B8610EE004F0AEF801F09EFD04F06EF8C1
:1018A0007861A86F04F0A6F801F008FE04F066F86D
:1018B000B861A87D0128BBD1786904F09BF801F0DC
:1018C0003DFE04F05BF87861B86904F093F801F02C
:1018D00073FE04F053F8B861AAE70000002C014041
:1018E0000000002028020020000801402001002004
:1018F00030B526486FF001010160254B25481A7864
:10190000102A1BD293F82A10012908D002290BD0E3
:1019100003290ED0016841F44001016012E0016822
:1019200041F0400101600DE0016841F0800101607B
:1019300008E0016841F0C001016003E0016841F482
:1019400040010160521CD1B200201970202900D141
:101950001870197E91B1104A1978104D52F8214033
:101960002D682C44A4F2FB7442F82140D96C491C28
:10197000D9641A6D914201D31876D8640748443867
:10198000016841F48001016030BD00001004004096
:101990000000002010080140280200204C240140D3
:1019A00070B50820FFF7DAFD234A82F823000520EE
:1019B000FFF7D4FD82F821000620FFF7CFFD9077D6
:1019C0001D49D07F0823803148F20104012814D03A
:1019D000022815D048F20F05032816D00A2604283D
:1019E00017D00423052819D006281DD0072803D1B5
:1019F00049F6DF004863D67470BD4C63D37470BD84
:101A000048F21F004863D37470BD4D630220D07448
:101A100070BD48F25F004863D67470BD4C63D374E8
:101A2000002082F8230070BD4D63D37406209077A8
:101A3000012082F8210070BD000000202DE9F04750
:101A4000F84D00242C71F84801680906FCD5F648C9
:101A5000001D006800F0FF090223B9F1410F2BD0EF
:101A6000E879002826D00126F04A44F60C610328C4
:101A700001D0022822D095F8300036287DD03528B4
:101A80007CD05A287BD056287AD0492879D047284C
:101A900078D0482877D0632876D0422875D061283E
:101AA00074D0742873D0782872D03D2871D07328F0
:101AB00070D0EC71BDE8F087EB71FBE7D94F803750
:101AC000B9F1440F74D0B9F1570F65D0B9F1450F92
:101AD0007ED0B9F1760F7CD0B9F1530F7AD04FF0A8
:101AE000140AB9F1540F76D0B9F1460F74D04FF4FF
:101AF0009670B9F12D0F70D0B9F1330F6ED0B9F1E6
:101B0000340F6CD0B9F1770F6AD0B9F16E0F68D08D
:101B1000B9F1710F66D0B9F17A0F71D04FF0030CA3
:101B2000B9F1720F6DD0B9F1620F6BD0B9F1500FEE
:101B300069D0BF4AB9F1660F7ED0B9F1670F7CD08A
:101B4000B9F1680F7AD04FF4B478B9F16B0F76D051
:101B5000B9F16A0F74D0B9F16C0F72D0B9F1650F99
:101B600070D0B9F1640F6ED0B24FDFF8CC824FF075
:101B70006636B9F1390F67D00FE022E22CE263E25A
:101B800076E279E286E290E296E29CE2A2E2A8E2C4
:101B9000B0E2B6E2B9E20BE036E0B9F1380F7DD041
:101BA000B9F1370F7BD085F807C085F8309081E711
:101BB0002A20FFF7FDFC287AFFF7FAFC687CFFF784
:101BC000F7FCB888C0F38710FFF7F2FCB8890AE089
:101BD00075E0C5E0D0E0DBE0E6E0F1E0FBE0FEE050
:101BE00001E10EE111E1C0F38710FFF7E1FC95F888
:101BF0003300FFF7DDFC0A20FFF7DAFCEC7159E750
:101C000007E10AE124E128E14020FFF7D1FC00F0E0
:101C100085FAC0B2FFF7CCFC10350F21A86BB0FBE2
:101C2000F1F0C0B2FFF7C4FC287EFFF7C1FCA87C2E
:101C3000FFF7BEFCA87D08E014E11DE127E12BE1E0
:101C400034E13DE140E14EE162E1FFF7B1FCE87AC9
:101C5000FFF7AEFC15F80E0CFFF7AAFC15F80D0CFB
:101C6000FFF7A6FC15F80D0CFFF7A2FCA87BFFF709
:101C70009FFC287FFFF79CFC687CFFF799FC687E3F
:101C8000FFF796FCA87AFFF793FCE87EA97E00EBAD
:101C90004100C0B2FFF78CFCE87B01E056E173E144
:101CA000FFF786FC97F84C00FFF782FC287CFFF7D3
:101CB0007FFC0A20FFF77CFC05F8094CFAE623209C
:101CC000FFF776FC95F82300FFF772FCA87CFFF77E
:101CD0006FFC686C5949401CB1FBF0F04009386456
:101CE00042F21076B0FBF6F0C0B2FFF761FC386C40
:101CF000B04201D3801B3864386C6426B0FBF6F028
:101D0000C0B2FFF755FC386CB0FBF6F106FB1100D2
:101D1000FFF74EFC386A90FBF6F0C0B2FFF748FCC4
:101D2000386A90FBF6F106FB1100C0B2FFF740FCE9
:101D3000A87DFFF73DFC287DFFF73AFC0320FFF765
:101D40001BFCFFF735FC0520FFF716FCFFF730FC06
:101D5000A87BFFF72DFC0A20FFF72AFCEC71A9E60F
:101D6000304837A239A1E030FEF736FA2D48E0308E
:101D700002F096FDEC719DE695F82200401E10F0F1
:101D8000FF0085F8220001D185F82260EC7191E610
:101D900095F82200401CC0B285F82200142801D911
:101DA00085F822A0EC7185E695F82800401CC0B2A9
:101DB00085F82800032801D985F82860EC7179E6B8
:101DC0004FF48071516101F0F7F941F2883001F070
:101DD00033FEEC716EE6AE75EE75EC716AE6AC75CD
:101DE000EE75EC7166E672B6A878022802D1012081
:101DF00000F0B0F962B6EE75C820FEF7BFFFEC71D7
:101E000058E6EC76EE75EC7154E6EE76EE75EC7114
:101E100050E6EB76EE75EC714CE685F81BC0EE757E
:101E2000EC7147E60000002000480040000C014033
:101E30002C04004066A64C400000F03F00B4C404EF
:101E400030312E30322E3236000000002573000073
:101E50004FF480501061EC712CE6322001F0ECFD63
:101E6000EC7127E6686C892803D9401E686410600D
:101E7000E963EE75EC711DE6686CB0F59B7F03D8E5
:101E8000401C68641060E963EE75EC7112E601F0C5
:101E900035F9EE75EC710DE6386A401E386201D5F1
:101EA000C7F82080FFF794FBEC7103E6386A401C0A
:101EB0003862404500DB3C62FFF78AFBEC71F9E5D4
:101EC00001F0B0F8EC71F5E501F076F9386AB4305C
:101ED000401C3862404502DBA0F5B4703862FFF761
:101EE00077FBEC71E6E507200D356874EE776B77CC
:101EF0002E752B776E7385F819A06C72AE74122054
:101F000068750620A8755620687105F8064CD1E55D
:101F1000A87C401C40B2A8745A2801DD5A20A8743D
:101F200095F91200404203F0CEF832463B4602F0EB
:101F3000D9FE02F013FD02460B460020414602F096
:101F4000D1FE02F0E1FD2864EC71B3E5A87C401EEF
:101F500040B2A874462801DA4620A87495F9120008
:101F6000404203F0B0F832463B4602F0BBFE02F0BE
:101F7000F5FC02460B460020414602F0B3FE02F09B
:101F8000C3FD2864EC7195E500F06CF9642001F064
:101F9000CDF92420FFF70CFB0320FFF7EDFAFFF744
:101FA00007FB0520FFF7E8FAFFF702FBA87BFFF726
:101FB000FFFAA878FFF7FCFA0A20FFF7F9FAEC71AC
:101FC00078E5EE75A87802288CD002F061FA4FEA25
:101FD00009202866EC716DE5A878022897D0286E54
:101FE00040EA09002866A87B401C40B2A873062876
:101FF00000DDFEE701F028F928792874A878022886
:102000001FD02C66EC73012000F0DEF82420FFF7CF
:10201000CFFA0320FFF7B0FAFFF7CAFA0520FFF75F
:10202000ABFAFFF7C5FAA87BFFF7C2FAA878FFF76B
:10203000BFFA0720FFF7BCFA0A20FFF7B9FAEC71E4
:1020400038E55520E873DEE785F814900820B9F1EB
:10205000580F0AD050616E7547F2305001F066F9A2
:10206000287D02F029FBEC7124E56C751061FAE71C
:1020700085F82690EC711DE5B9F10B0F08D209F037
:10208000010085F82B004FEA590085F82A00E96322
:10209000EC710FE5B9F1030F01D285F8219095F8A5
:1020A0002100FEF773FAEC7104E5B9F10B0F01D2D0
:1020B00085F81E90EC71FDE4B9F1050F01D285F8A9
:1020C0002C90EC71F6E4B9F1050F01D285F8299056
:1020D000EC71EFE4B9F1060F01D285F81A90EC71BA
:1020E000E8E4B9F1080F01D285F81F90FFF758FC1A
:1020F000EC71DFE4B9F10A0F01D285F82390EC719D
:10210000D8E485F82090EC71D4E4B9F1030F01D242
:1021100085F8039001F08EFAEC71CBE400B50B4921
:1021200000200860142001F001F908483438816863
:1021300041F4A00181600168C1F340010029FAD097
:10214000C06C80B24E21B0FBF1F000BD34280140DC
:10215000FEE7000070B5012801D102F07BFC1648B3
:102160001449416015494160154800F04DF8144C80
:10217000144DE41EE078404205EBC020FEF778FBEA
:10218000E0781022404205EBC02104F1ED00FEF79B
:102190008DFBE0780B494042103101EBC021102249
:1021A00004F1FD00FEF782FBBDE870403220FEF72F
:1021B000E5BD00002301674500200240AB89EFCD5B
:1021C0000300002000FC010810B50B49094A4A60D1
:1021D0000A4A4A60012801D102F080FC084C2046DE
:1021E000FEF746FB2146BDE8104008220548FEF7F1
:1021F0005DBB00002301674500200240AB89EFCDA5
:1022000000D40108E500002010B5054C2046FEF77B
:102210002FFB2146BDE8104002220248FEF746BBD4
:1022200000DC01080300002070B506460D46FEF7ED
:1022300087FA4FF47A74204601F078F85820FEF7B8
:10224000BBFA204601F072F83046FEF7B5FA204698
:1022500001F06CF82846FEF7AFFABDE87040FEF7D3
:1022600095BA000010B50320FFF786F9FF282DD09E
:1022700000220320FFF780F950B3002002432DD045
:102280000520FFF779F9FF2824D000220520FFF769
:1022900073F908B30020024320D0FEF789F9104BF0
:1022A000D86503F1E50166224A7000228A709A73AC
:1022B000040ACC7048710A718A711A6693F8480052
:1022C000C871BDE810400020FFF77EBF0122D0E7B3
:1022D0000120D3E70122D9E70120DCE710BD00008F
:1022E00000000020490050EAC12018BF04204A0D18
:1022F00018BF40F0010040F2FF72B2EB515F08BF1F
:1023000040F00200012808BF0520704700280DDBBF
:1023100000F01F02012191404009800000F1E020FF
:10232000C0F88011BFF34F8FBFF36F8F7047002845
:1023300009DB00F01F02012191404009800000F1FB
:10234000E020C0F80011704702480068C0F3022086
:10235000704700000CED00E00907090E002804DBBF
:1023600000F1E02080F80014704700F00F0000F149
:10237000E02080F8141D70470907090E002804DBCF
:1023800000F1E02080F80014704700F00F0000F129
:10239000E02080F8141D70472DE9F74F144694B0E3
:1023A0000021C4E902111599079121F00045C9499E
:1023B0008D4206DC1599C4E9000117B00020BDE884
:1023C000F08FC549DFF814A3A9423CDD0799C44E3C
:1023D0000029C44FC44A1599534619DD03F08EF8FD
:1023E000554506D0C14AC24B03F088F8C4E9000144
:1023F0000AE04FF0D352BE4B03F080F832463B4622
:1024000003F07CF8C4E9000117B00120BDE8F08FAB
:1024100002F0ACFB554506D0B44AB54B02F0A6FB22
:10242000C4E900010AE04FF0D352B14B02F09EFB29
:1024300032463B4602F09AFBC4E9000117B04FF068
:10244000FF30BDE8F08FAB49A942159978DB21F048
:10245000004183468846A84AA84B02F05FFE00224E
:10246000A74B02F083FB02F0D1FD099002F02BFE96
:1024700006460F469C4A534602F050FE43465A46D3
:1024800002F04AFF80468A46984A994B30463946C0
:1024900002F044FE2A0D01250B924246534602F0FB
:1024A0003BFF032DC4E9000139D00B98C1F30A5159
:1024B000401A05EB45111139814230DA9148C34683
:1024C000784400EB0510CDF80CA00C90D0E9002367
:1024D0003046394602F022FE02460B460491069031
:1024E0005846039903F00AF880468A4602460B468E
:1024F0005846039903F002F8049B069A02F0FEFF87
:1025000083460C9803913946D0E90223304602F005
:1025100005FE5A46039B02F0F1FF6D1CBDE70798CC
:102520000028A2BF099817B0BDE8F08F616881F05C
:1025300000416160099817B04042BDE8F08FFFE7A5
:1025400084461598C1F31301C0F30A50A0F2F53088
:102550004FEA601800F01F06C6F12000139000201B
:102560000690079041F4801E05206D4676B1664ABC
:1025700008EB00017A4452F8213002EB8101B340AC
:102580004A68139922FA01F1194305E05F4908EB03
:102590000002794451F82210A1FB0E27A1FB0C1375
:1025A0001A449A4234BF0123002303EB070A05EBC8
:1025B0008003D3E901B70F448F4234BF01210021CA
:1025C00093448B4411B1934502D903E0934501D262
:1025D000012100E00021C3E901B7514445F8201072
:1025E000011EA0F10100C1DC0298059F00F100501E
:1025F000800F12900298DDE90356800002F063FD1F
:10260000834628460D9102F075FD6FF01D0203F020
:1026100090FBCDE90E01304602F06CFD6FF03D02FB
:1026200003F087FB80468A46384602F063FD6FF070
:102630005D0203F07EFB074642465346119102F0CD
:1026400095FADDE90E2302F091FA5A460D9B02F04D
:102650008DFA00250E465A4628460D9B02F04EFF85
:10266000DDE90E2302F04AFF4246534602F046FFE0
:102670003A46119B02F050FEDFF898A0244A5346D8
:1026800002F04CFD07468846234A244B3146284633
:1026900002F044FD3A46434602F068FA074688468F
:1026A0004FF0A84253463146284602F037FD3A46DD
:1026B000434602F05BFA159A12F0004F04D0129ACA
:1026C00081F0004152421292C4E90001129817B001
:1026D000BDE8F08FFB21E93F7CD90240FB21F93FA7
:1026E0007370032E8A19A33B000040543163621AB1
:1026F00061B4D03DFB21394183C8C96D305FE43FEF
:102700000000E03F243B0000A03A0000823A0000B5
:10271000182D4454FB21F93D3326A611460B113CDC
:102720002DE9FF4D21F0004807460C46B8F1795FCE
:1027300008DA02F06BFC002801BF0020324904B027
:10274000BDE8F08D3A4623461046194602F0E6FCF5
:10275000054602462D480E460B460621784400F0F9
:102760005DF82A46334602F0D9FCDDE902238246B1
:102770008B463846214602F0D1FC04460F465246AD
:102780005B462846314602F0C9FC22463B4602F031
:10279000B5FE07468A464FF0FF322846314603F021
:1027A000C8FA1B4A90450ADA3A46534602F0A6FE9A
:1027B00004B00022BDE8F04D134B02F0ADBD154A48
:1027C0004245A8BFA8F500154FF00004B8BF124D50
:1027D00022462B4602F092FE0646884622462B46AB
:1027E0000020094902F08AFE04460D463A46534647
:1027F0003046414602F082FE04B022462B46BDE838
:10280000F04D02F089BD00000000F03F503800009C
:102810003333D33F0000E93F0000D23F2DE9F041C0
:102820004F1E00EBC7010446D1E9000115461E46C4
:1028300037F006020DD02A46334602F06FFC7F1EA9
:1028400004EBC703D3E9002302F090F937F0060246
:10285000F1D1022F25D0042F13D0062F18BFBDE8C9
:10286000F0812A46334602F059FCD4E90A2302F0EB
:102870007DF92A46334602F051FCD4E9082302F0E0
:1028800075F92A46334602F049FCD4E9062302F0E2
:102890006DF92A46334602F041FCD4E9042302F0E4
:1028A00065F92A46334602F039FCD4E9022302F0E6
:1028B0005DF92A46334602F031FCD4E90023BDE835
:1028C000F04102F053B900002DE9FF4D054621F01B
:1028D000004084B00C46B0F1795F0BDA2846FFF770
:1028E00001FD042808BF00F0B7F9284608B02146CA
:1028F000BDE8F08D2A460B46104602F00FFC064656
:102900000F462A46234602F009FC804626488A469E
:1029100032463B4605217844FFF780FF83461098F6
:10292000029160B3214A224B4046514602F0F6FB29
:10293000CDE900015A4640465146029B02F0EEFBAB
:1029400082468846DDE906014FF0FF3203F0F1F9D7
:102950005246434602F0D2FD32463B4602F0DEFBD1
:10296000DDE9062302F0CAFDDDE9002302F0C6FD21
:1029700008B02A462346BDE8F04D02F0CDBC0B4618
:102980005A463046394602F0C9FB084A084B02F065
:10299000EDF84246534602F0C1FB08B02A462346F2
:1029A000BDE8F04D02F0E2B89637000049555555A4
:1029B0005555C5BF2DE9F04D04468CB0904821F027
:1029C0000047164698460D460991874206DA20468A
:1029D000294602F01BFB002800F0AE808948B8426F
:1029E0001CDC09980028BCBF85F0004588F0004831
:1029F000854A864B2046294602F08EFC04460D4649
:102A0000324643468248834902F078FD22462B46EF
:102A100002F0ACF8002604460D46B04622462B468E
:102A20001046194602F07AFB8B46824602460B4658
:102A300002F074FB0246089077480B46009106218D
:102A40007844FFF7EBFECDE9031074480621784483
:102A5000009B089AFFF7E2FE52465B4602F05EFBDF
:102A6000CDE9051052465B462046294602F056FB4A
:102A700007910090DDE90310DDE9053202F076F8F8
:102A8000079B009A02F04AFB3246434602F06EF87A
:102A900052465B4602F042FB3246434602F066F87D
:102AA00080460E465E4A5F4B0799009802F036FB5F
:102AB0004246334602F05AF882468B4622462B465F
:102AC00002F054F880464F480E46B84214985BDC3A
:102AD00002F0F9FA074642463346059102F046F8FD
:102AE000CDE90110424633461046194602F016FB66
:102AF000DDE9013202F0F6F852465B4602F0FEFCD8
:102B000022462B4602F008FC012203F012F93A4655
:102B1000059B02F001FC04460D460998022101EADA
:102B2000A070C0F1010002F0CEFA0CB022462B4694
:102B3000BDE8F04D02F0F2BA1498401C384320432F
:102B40000BD01498012812D00CB022462B46BDE8B9
:102B5000F04D0020344902F0C5B80CB025F0004318
:102B60002246BDE8F04D0020304902F0BBB82046B7
:102B70002946FFF7B7FB042808BF00F06DF8204690
:102B80000CB02946BDE8F08D012802BF40460CB0CC
:102B9000BDE8F08D00270B463A462046294602F054
:102BA000BBFB52465B4602F0B7FB04460D4642466D
:102BB000334600201C4902F095F883463A46884681
:102BC0003346104602F0AAFA0022184B01F0CEFF5D
:102BD00006468A4622462B463846414602F09EFA71
:102BE0003246534601F0C2FF5A46434602F096FA77
:102BF0000CB03A464346BDE8F04D01F0B7BF0000C7
:102C00000000303E2894E53F182D4454FB21E93F55
:102C1000075C143326A6813C94360000B6360000CB
:102C2000635555555555D53F0000F0BF0000F03FA6
:102C3000002213461046014902F054B80000F03F4C
:102C4000012203F076B801F091BF0022134610462E
:102C5000114602F047B80000024A0020110703F0B5
:102C600068B8000001FDFFFF2DE9F84F04460D464E
:102C700021F0004000917349814211DC7249884281
:102C800001DC06D12CB120462946BDE8F84FFFF7FC
:102C9000D7BF6E48002DCCBF6D496E49BDE8F88F97
:102CA0006D49814211DD6D498142D8BF4FF0FF3639
:102CB0006DDD20462946FFF715FB042808BFFFF706
:102CC000CBFF20462946BDE8F88F6549654F25F0C2
:102CD0000045814233DD6449814219DD00263246D8
:102CE0004FF080432046294601F040FF80468A4647
:102CF00001222046294603F01CF800223B4602F040
:102D0000FDFB4246534601F0EDFF04460D463EE012
:102D100001260022BA463B462046294601F026FFFE
:102D200080460F46002253462046294602F0E6FB25
:102D300042463B4601F0D6FF04460D4627E04B498C
:102D400081421BDDDFF828A10226002253462046DF
:102D5000294602F0E3F900223B4601F007FF8046D6
:102D60000F46002253462046294602F0C7FB424642
:102D70003B4601F0B7FF04460D4608E00326224615
:102D80002B4600203B4901F0ADFF04460D4622468C
:102D90002B461046194602F0C1F98B468246024680
:102DA0000B4602F0BBF907460246334888460B46FD
:102DB00006217844FFF732FD52465B4602F0AEF939
:102DC00082462E488B463A46434605217844FFF713
:102DD00025FD3A46434602F0A1F902460B46002E75
:102DE000504659460CDA01F0C1FE22462B4602F04D
:102DF00095F901B022462B46BDE8F04F02F08CBA9F
:102E000001F0B4FE22462B4602F088F91C4A7A44AF
:102E100002EBC603D3E9002302F070FB22462B46E7
:102E200002F06CFB174A7A4402EBC603D3E9002395
:102E300002F072FA009A002AB8BF81F00041BDE8A2
:102E4000F88F0000000010440000F07F182D44545B
:102E5000FB21F93FFB21F9BF0000DC3F0000203ED1
:102E60000000F33F0000F03F0000E63F0080034019
:102E70000000F83F0000F0BFCA31000088310000B8
:102E800026310000EE3000002DE9F04D9446CCF1E3
:102E9000000423F000464CEA0404594F46EAD47477
:102EA0009A46884621F00042BC4206D8454240EA94
:102EB000050442EAD474BC4204D9BDE8F04D624630
:102EC000FFF7C1BEAAF14055A5F17F6555EA0C0494
:102ED0000BD0022404EAAA744A4DDFF82CE144EA3C
:102EE000D87452EA000B04D00CE0BDE8F04DFFF7B7
:102EF000BBBE002C14BF012CBDE8F08D022C30D0DD
:102F0000032C32D056EA0C0B0AD0BE4220D1BA4272
:102F100009D126F0804622F080423346114617E060
:102F200000291ADB25E0DFF8E4B0FB44002C04BFE5
:102F3000DBE90001BDE8F08D012C02BFDBE90001F7
:102F400081F00041BDE8F08D022C0AD0032C0CD09A
:102F5000BA4212D1B8F1000F0BDA2A482C49BDE869
:102F6000F08D28462B49BDE8F08D28467146BDE816
:102F7000F08D24482849BDE8F08D921B12153C2A9B
:102F8000C4BF204F244E10DCBAF1000FBEBF12F1B7
:102F90003C0F00273E4608DB624601F0A3FE21F00D
:102FA0000041FFF761FE07460E4694B1012C08BFB1
:102FB00086F000460DD0194A194B022C384631468E
:102FC00015D002F09BFA2A46BDE8F04D114B02F0F5
:102FD00095BA002213463846314601F0DBFF04BFA4
:102FE0000220FDF7FEF938463146BDE8F08D02F0CB
:102FF00085FA2A46BDE8F04D064B02F08DB9000077
:103000000000F07F182D4454FB2109C0B2300000AD
:10301000FB21F9BFFB210940FB21F93F075C143379
:1030200026A6A13C2DE9F047DFF8C080D8F80000C3
:1030300020F02000C8F800004FF08040016821F027
:1030400001010160C1132A4841612A4F0020386202
:10305000FEF7BEFA40F2DC50FDF790FEA7F18006C5
:103060000120F0754FF4167000F0A6F84FF4FA60E6
:10307000FDF784FE00250024B06F02F0BBFC814602
:10308000706F02F0B7FC494601F0CCFC05446420A7
:1030900000F0D2FC641CE4B2142CEDD3142095FB98
:1030A000F0F0154A4AF6AA2111605A3040423862BF
:1030B000B0F5B47F02DDA0F5B4703862386A00283C
:1030C00002DA00F5B4703862FEF782FA642000F08C
:1030D000B3FCD8F8000040F02000C8F80000BDE8BC
:1030E000F0474FF47A7000F067B800000C480040D9
:1030F0000008014080000020003000402DE9F04130
:1031000000244FF08040016821F00101016017495F
:10311000C0134861164D8920686440F23711A964D4
:103120002864A5F18006134F0DE03860282000F0D8
:1031300083FCFDF76DFBA04202DD0446286C706441
:10314000286C401C2864A96C286C8842EDD3FEF7DB
:1031500081F909494AF6AA200860502000F02CF8AD
:1031600044F60C60F063BDE8F08100000008014007
:10317000800000202C040040003000400C4A92F8EF
:1031800027204A43D1B2002900D10121C82900D902
:10319000C821782800D27820064AB2FBF0F24FF01E
:1031A0008040C2620164016841F001010160704722
:1031B0000000002038A2870070B50E4E4FF4004585
:1031C00035610D49EC03B1FBF0F0E0620B4890F87B
:1031D0002600410841432164206840F0010020603E
:1031E0008220FDF7CBFD206820F001002060756192
:1031F00070BD00000008014038A2870000000020D8
:10320000F0B5044608220E4D0E4ED3064EF660274A
:10321000186840F00100186095F82610491C5143C9
:103220001964B6FBF4F0D862384600F07FF81868ED
:1032300020F001001860521E002AE9DCF0BD0000F9
:103240000000002038A2870070B50520FEF794F931
:1032500002460320FEF790F90C4C42EA0020E0659C
:1032600000F052F9216E01260425884209D1FDF7AC
:103270009FF9E16D884204D184F82E500220A0709D
:1032800070BD84F82E50A67070BD000000000020B4
:1032900000B5244B21F0004287B09A42DCBF0022E7
:1032A000134629DD204B9A4208D140B94FF0010066
:1032B000FDF797F8FFF7C9FC07B000BD03DBFFF788
:1032C000BFFC07B000BD02AAFFF766F810F00301CB
:1032D00004BF0DF1080C9CE80F000DD0012001295E
:1032E0000ED0022914D00DF1080C00909CE80F00BC
:1032F000FFF7EAFA07B000BDFFF712FA07B000BD0A
:103300000DF1080C00909CE80F00FFF7DDFA05E0D6
:103310000DF1080C9CE80F00FFF702FA07B081F0EE
:10332000004100BDFB21E93F0000F07F0146491E3E
:10333000FDD10146491EFDD14008401EFDD1704718
:103340002DE9F041014600250A240E4E621E56F872
:10335000220046F82400D4B2002CF7D131600A4F85
:1033600056F8241057F8240002F070FB294602F0AA
:10337000DBF90546641CE4B20B2CF1D32846BDE80A
:10338000F081000030030020305E00082DE9F0419C
:103390000146002508240E4E621E56F8220046F80B
:1033A0002400D4B2002CF7D131600A4F56F8241013
:1033B00057F8240002F04AFB294602F0B5F9054609
:1033C000641CE4B2092CF1D32846BDE8F08100006A
:1033D000880300205C5E00082DE9F04101460025CD
:1033E00006240E4E621E56F8220046F82400D4B27F
:1033F000002CF7D131600A4F56F8241057F82400FA
:1034000002F024FB294602F08FF90546641CE4B261
:10341000072CF1D32846BDE8F0810000D00300203E
:10342000805E00082DE9F041014600250A240E4E79
:10343000621E56F8220046F82400D4B2002CF7D1C0
:1034400031600A4F56F8241057F8240002F0FEFAB3
:10345000294602F069F90546641CE4B20B2CF1D34D
:103460002846BDE8F08100005C030020305E0008C3
:103470002DE9F0410146002508240E4E621E56F843
:10348000220046F82400D4B2002CF7D131600A4F54
:1034900056F8241057F8240002F0D8FA294602F012
:1034A00043F90546641CE4B2092CF1D32846BDE873
:1034B000F0810000AC0300205C5E00082DE9F041C3
:1034C0000146002506240E4E621E56F8220046F8DC
:1034D0002400D4B2002CF7D131600A4F56F82410E2
:1034E00057F8240002F0B2FA294602F01DF9054609
:1034F000641CE4B2072CF1D32846BDE8F08100003B
:10350000EC030020805E000870B5C0F30725C4B24C
:10351000284601F0EFFD00F0E1F805FB045104F14D
:1035200008000844C4F1FF010144091DC9B24FF667
:10353000FF7202EA0020084470BD00002DE9F04748
:1035400003211A4EA6F110054A1E56F8223046F8FD
:10355000213055F8223045F82130D1B20029F3D17D
:103560003060134902F072FA28600124DFF84480C9
:10357000A8F1100955F8241058F8240002F066FA52
:10358000074656F8241059F8240002F05FFA39462D
:1035900002F028FB296802F0C7F82860641CE4B236
:1035A000032CE7D92868BDE8F08700009C040020C0
:1035B0005BC0FF3CAC5E00082DE9F04703211A4ECA
:1035C000A6F110054A1E56F8223046F8213055F86B
:1035D000223045F82130D1B20029F3D130601349AF
:1035E00002F034FA28600124DFF84480A8F11009C1
:1035F00055F8241058F8240002F028FA074656F827
:10360000241059F8240002F021FA394602F0EAFAAF
:10361000296802F089F82860641CE4B2032CE7D919
:103620002868BDE8F0870000BC0400205BC0FF3CB8
:10363000AC5E000810B500F02BFFFDF70BFFFEF7A6
:10364000AFF90E4C94F91200404201F03CFD4FF0EE
:1036500066320B4B01F046FB01F080F902460B4647
:103660000020084901F03EFB01F04EFA206494F876
:103670002100BDE81040FCF789BF000000000020D9
:1036800066A64C400000F03F2DE9F04180460C4614
:10369000C2F10B0002F0AEF90E4902F0ADF805469A
:1036A00029464FF07E5002F09DFA0B4F57F8241038
:1036B00002F0CCF906462946404602F0C7F93146E9
:1036C00002F032F847F8240002F058F9BDE8F04162
:1036D00002F090B90000F041080400202DE9F04DFF
:1036E000C84A002490B0914205DA21F00043934289
:1036F00001D805D120B110B0BDE8F04DFFF7A0BA58
:10370000B1F5801F1BDA53EA000209D0002911DA53
:103710000120FCF766FE10B0BDE8F04DFFF795BA4A
:103720000220FCF75EFEFFF783FA10B081F0004143
:10373000BDE8F08D6FF03504362202F0FAFA04EBA2
:103740002152C1F31308B049A2F2FF33414401F4FE
:10375000801282F07F6103EB225281F0405100928F
:1037600041EA08010022A94B01F0C8FE044608F115
:103770000200A74EC0F313000D467E44032867D213
:10378000D6E90023204601F005FC1ED10098002850
:1037900002BFD6E9000110B0BDE8F08D01F093FC46
:1037A00007460C469B4A9C4B01F0B8FC06460D466A
:1037B0009A4A9B4B3846214601F0B0FC10B0324685
:1037C0002B46BDE8F04D01F0D1B94FF05532954B85
:1037D0002046294601F0A2FC0022934B01F09CFDFB
:1037E00006460F4622462B461046194601F096FC27
:1037F00032463B4601F092FC064600980F46F0B177
:1038000001F061FC80468A46824A834B01F086FCC7
:1038100032463B4601F080FD22462B4601F06EFE0B
:1038200005460C467D4A7E4B4046514601F076FCEB
:1038300010B02A462346BDE8F04D01F05FBE0B46AE
:1038400010B0324620462946BDE8F04D01F056BE84
:1038500000224FF08043204601F088F902460B46D3
:103860002046294601F03EFA06460F46009801F030
:103870002AFCCDE9040132463B461046394601F0A8
:103880004DFC0C9069480C9A4044019009910B46FC
:10389000104601F043FC8246024665488B46C8F15B
:1038A00051080B4608F5D72803217844FEF7B6FFE8
:1038B00052465B4601F032FC0A905E480D9152463A
:1038C0005B4604217844FEF7A9FF099B0C9A01F09E
:1038D00025FC844601980D9B40EA080860460A9A38
:1038E00001F044F983460891B8F1000F4EDD4FF026
:1038F000FF322046294602F01CFA22462B4601F0F0
:103900000DFC804600988A4660B3DDE90401414A17
:10391000414B01F003FC099100905A464046514644
:10392000089B01F023F932463B4601F0F7FB099B67
:10393000009A01F01BF94246534601F0EDFC224685
:103940002B4601F0DBFD04460D46DDE90401334A58
:10395000334B01F0E3FB10B022462B46BDE8F04D9F
:1039600001F0CCBD5A464046089B01F0FFF83246B4
:103970003B4601F0D3FB4246534601F0CDFC10B06C
:1039800022462B46BDE8F04D01F0C6BC009840B37E
:10399000DDE904011F4A204B01F0C0FB80468A4646
:1039A0005A4620462946089B01F0A8FD32463B4670
:1039B00001F0B4FB4246534601F0A0FD22462B46DF
:1039C00001F09CFD04460D46DDE90401134A144B49
:1039D00001F0A4FB10B022462B46BDE8F04D01F0EB
:1039E0008DBD0B465A462046294601F087FD3246DA
:1039F0003B4601F093FB10B022462B46BDE8F04D4C
:103A000001F08ABC0000F07F645F09000000F03F15
:103A100062280000763C7935EF39EA3D0000E0FE8F
:103A2000422EE63F5555D53F0000E03F86EBF9FFBB
:103A30003226000030260000FDF7A0B91CB5FCF7C7
:103A4000EDFDFDF7D3FDFDF74BFAFDF7A7F9FDF707
:103A5000F9F9FDF781FBFDF7DBFAFDF715FBFDF743
:103A6000A7FAFDF7B1FBFDF7B9FA6420FFF7E4FF11
:103A7000F94D4FF4807028616420FFF7DDFF72B6C6
:103A8000F648416821F0E06141F000714160F44E78
:103A9000B06840F00100B0601E20FDF76FF9B0681B
:103AA00040F00400B060B068C0F380000028FAD095
:103AB000EC4EB06840F00100B0601E20FDF75EF9EA
:103AC000B06840F00400B060B068C0F38000002827
:103AD000FAD0E3480830016841F480110160E248FF
:103AE000016821F002010160C16841F00101C1607B
:103AF000011D0A6842F020020A60016841F00101DC
:103B0000016081140005026A42F480520262D748C3
:103B1000026822F002020260C26842F00102C26042
:103B2000026842F0010202606961D148016841F017
:103B30000C010160016841F020010160001D4FF09F
:103B4000000AC0F800A0001DC0F800A06420FFF724
:103B500073FF0020FDF702FDC64EFF2815D101209E
:103B6000FDF7FCFCFF2810D186F803A00020FEF72B
:103B7000F1FAF078401CC0B2F0700428F6D386F851
:103B800003A0BC48C01CFEF73FFB86F82FA0FDF742
:103B9000FFFCF0704FF00109012801D986F803906D
:103BA000FFF748FD86F83590707D01287ED008200B
:103BB000286162B64FF4FA70FDF7E0F886F81790C6
:103BC000C820FDF7DBF8AC4F4FF4004038614FF4EC
:103BD000804BC5F810B040F6AC50FFF711FB142035
:103BE000FDF7CCF89C494FF4004008614FF4FA60AF
:103BF000FFF706FB1420FDF7C1F897484FF4005873
:103C0000C0F810804FF47A70FFF7FAFA3220FDF70F
:103C1000B5F89148C0F814804FF4C860FFF7F0FA87
:103C20008D494FF4004048611420FDF7A7F88A48F9
:103C3000C0F814B04FF400407861FFF705FB8D48E1
:103C40008EA291A1E030FCF7C7FA8A48E03000F07C
:103C500027FE4FF0000800214FF4B0420846FDF760
:103C600093FC8044091D9142F8D3B06B804526D067
:103C70004FF47A70FFF7A0FA4FF47A60FDF77EF800
:103C80004FF4FA70FFF798FA7A48424680A1E03084
:103C9000FCF7A2FA7748E03000F002FE41F28830EB
:103CA000FFF7CAFE20206861FEE7FFE70820686191
:103CB0006420FFF7C1FE307D00F0FEFC79E7DFF8FD
:103CC000B48196F8210008F18008A8B1D8F828003E
:103CD000C8F82000FDF77CFC6420FFF7ADFEFEF77E
:103CE0001DFA42F21070FFF721FB41F21001624809
:103CF000FCF75EFF28B114E0D8F82400C8F82000D3
:103D0000E8E74FF47A70FFF757FA4FF4FA70FFF7CD
:103D100053FA5848C17E59B380F81BA0C820FDF75C
:103D20002DF8544D2035A878C0F11400A87405F181
:103D30006008EE6CC8F80460296DC8F80C10019199
:103D4000304601F057FE296A01F080FE07460198CF
:103D500001F050FE394601F045FF01F00FFEC8F8B2
:103D60001C0015F8201931B17110C8F8301005E0A9
:103D700080F81B90D2E76421C8F83010C01C01F015
:103D8000A2F9FFF7ABFC01F041F9C8F82C000D28AF
:103D900002DD0D20C8F82C00E87E78B398F82C00DE
:103DA000801E687495F91100002801DA85F811A0C9
:103DB000D8F81C0047104CF25030874209DD06212C
:103DC0007820FFF7DBF949F64040FFF7AFFA85F8B6
:103DD00025A028481A30027B42730178052913D0A8
:103DE000D8F82C00234BC0F10E0592FBF5F202EB44
:103DF0004202D2B283F82720CAB11AE0FFE798F84E
:103E00002C00401E6874CDE700202349FFF766FCB4
:103E100005460E46D8F82C0001F055F92A463346DF
:103E200000F060FF01F022F91249487603E083F8C0
:103E30002790084458760F4D95F82500012809D1A0
:103E400085F825A0E87E30B101287DD002287CD0FD
:103E500003287BD00EE221E0000C0140000001406D
:103E6000002401400028014000040040002C0140D3
:103E70000C480040000000200008014030312E3086
:103E8000322E3236000000002A25732A200000005E
:103E9000256C6420000000000000104095F83200FE
:103EA000D8F81C1081423DDDD8F83010814239DD50
:103EB00085F81CA0687F401CC0B268770A2801D929
:103EC00085F81790D8E90101461AC8F80460D8E9C6
:103ED0000301401AC8F80C0001F08CFD0090304638
:103EE00001F088FD009900F06BFD40B22872687304
:103EF000D8F81C10A14203DDA872C8F838700C462F
:103F000095F90C10884200DAE872E87A2873A87AEA
:103F1000287295F82C10D8F82C0088429ADD00F011
:103F200055FBA7E14FF08040016821F001010160DD
:103F3000D8F80400C8F80800D8F80C00C8F8100039
:103F40005446C8F838A002E008E070E003E15A20C7
:103F5000E872287F401C28776C778BE195F8320057
:103F6000D8F81C10B1EBC00F3EDDD8F83010B1EB23
:103F7000C00F39DD85F81CA0687F401C6877D8E940
:103F80000101461AC8F80460D8E90301401AC8F8CC
:103F90000C0001F02FFD0090304601F02BFD009940
:103FA00000F00EFD41B22972D8F81C00A04203DDDA
:103FB000A972C8F838700446A87A2873287295F850
:103FC0002810082000EB4100697F884207D295F84D
:103FD0002C10D8F82C00884201DD00F00DFC4FF4C5
:103FE0007A70FFF7A3F945E14FF08040016821F0B6
:103FF00001010160D8F80400C8F80800D8F80C00E6
:10400000C8F810000024C8F838A05A20E87285F8D3
:104010001DA0287F401C2877FF484FF400414161D4
:10402000FE48C0F814B041614114416122E195F8A5
:104030003210D8F81C0088424CDDD8F83020B2EBA2
:10404000410F47DD322801DDC8F8589085F81CA0E3
:10405000687F401CC0B26877502801D985F8179056
:10406000D8E90101461AC8F80460D8E90301401AEA
:10407000C8F80C0001F0BEFC0090304601F0BAFC1C
:10408000009900F09DFC40B22872D8F85C10014401
:10409000C8F85C10D8F81C10A14203DDA872C8F85B
:1040A00038700C46A87A2873287295F828100820D2
:1040B00000EB4100697F884207D295F82C10D8F8B0
:1040C0002C00884201DD00F097FB4FF47A70FFF777
:1040D0002DF9CFE000204FF080410864D8F80400AB
:1040E000C8F80800D8F80C00C8F810005446C8F802
:1040F00038A0287F401C2877D8F85800012819D10B
:10410000687F142816D9D8F85C1091FBF0F2232AA6
:1041100004DD40F6B830FFF773F80BE091FBF0F0E8
:1041200010F1140F06DAE87F022803D04FF49670DE
:10413000FFF766F8C8F85CA0C8F858A085F81DA07D
:10414000B5484FF400414161B448C0F814B0416132
:10415000411441618EE095F83210D8F81C00884275
:104160004CDDD8F83020B2EB410F47DD322801DDBD
:10417000C8F8589085F81CA0687F401CC0B26877CA
:10418000502801D985F81790D8E90101461AC8F8D6
:104190000460D8E90301401AC8F80C0001F02AFCB9
:1041A0000090304601F026FC009900F009FC41B275
:1041B0002972D8F85C000844C8F85C00D8F81C00E4
:1041C000A04203DDA972C8F838700446A97A2973A1
:1041D000297295F82820082101EB42016A7F91425B
:1041E00007D295F82C20D8F82C10914201DD00F070
:1041F0002DFB4FF47A70FFF799F83BE0D8F80400F4
:10420000C8F80800D8F80C00C8F810005446C8F8E0
:1042100038A0287F401C2877D8F85800012819D1E9
:10422000687F142816D9D8F85C1091FBF0F2232A85
:1042300004DD40F6B830FEF7E3FF0BE091FBF0F051
:1042400010F1140F06DAE87F022803D04FF49670BD
:10425000FEF7D6FFC8F85CA0C8F858A085F81DA0E6
:104260006D484FF4004141616C48C0F814B04161A1
:1042700041144161287FC8287ED00020697FC82969
:104280007BD0002108430DD0C8F838A085F809A0DC
:1042900085F80DA085F808A085F811A085F817907D
:1042A00085F834A02F4695F90850DFF87481D8F8C6
:1042B0003800C01C00F007FFFFF710FA0022594B2E
:1042C00001F01CF900F0A2FE0646D8F83800C8F844
:1042D0003C00D8F81C003C284BDD7D7295FBF6F0C5
:1042E00000EBD070400887F8340097F90A0097F97E
:1042F0000C10401AC01C00F0E6FEFFF7EFF900F0CA
:1043000085FE97F8341091FBF0F0C0B287F83400C6
:10431000552D03DC97F90C10002902DA400887F8C4
:10432000340097F82D0000F13C018D4207DB44304A
:10433000854204DC97F83400400887F83400002EEA
:1043400001DA87F834A097F834000A2802D90A2045
:1043500087F8340097F83410B879091A01EBD17155
:1043600000EB610087F83400B871F54201D187F89D
:1043700034A097F8340001E058E059E087F83300A2
:10438000294E264D31462846FCF712FCD0B34FF497
:104390009670FFF751FB31462846FCF709FC88B3BD
:1043A000C5F810B04FF400462E614FF40058C5F820
:1043B00010804FF49670FCF7E1FC174806616E61BF
:1043C0004FF44870FEF7F8FE3220FCF7D7FCC5F832
:1043D00014804FF4FA70FEF7EFFE3220FCF7CEFCAB
:1043E000C5F814B04FF49670FEF7E6FE3220FCF7E5
:1043F000C5FC6420FEF7E0FEA815686141F2883034
:10440000FFF71AFB97F83100401C10F0FF0087F807
:1044100031000FD017E0000000080140000C0140FF
:10442000800000200000F03F02000204012025E788
:10443000012127E77878F0B14FF400562E611E2055
:10444000FCF79CFC6E61F96B44F6206081420DD94B
:10445000C7F83CA003207870FCF7DAF90A49C86471
:10446000B86CB0F57A7F01D287F8179007494AF601
:10447000AA20086035E4C5F810B01E20FCF77EFCC9
:10448000C5F814B0DFE700008000002000300040D5
:1044900000B51620FDF762F84B4A90750120FDF734
:1044A0005DF8107550750220FDF758F81072032062
:1044B000FDF754F8D0750420FDF750F8107605206C
:1044C000FDF74CF8D0730620FDF748F8107307206D
:1044D000FDF744F850730820FDF740F850740920A8
:1044E000FDF73CF890760A20FDF738F810700B20A5
:1044F000FDF734F890730C20FDF730F810710D20A3
:10450000FDF72CF890700E20FDF728F850770F205B
:10451000FDF724F890741220FDF720F803461120CF
:10452000FDF71CF843EA0020C2F83200123A5A287C
:1045300001D25A2050641420FDF710F8224B6E333C
:1045400058621320FDF70AF818B1586A00F5807018
:1045500058621A20FDF702F898621920FCF7FEFF56
:1045600018B1986A00F5807098621520FCF7F6FF84
:1045700082F822001720FCF7F1FF50751820FCF795
:10458000EDFFD0760120FCF7F7FFD0730220FCF797
:10459000F3FF90730520FCF7EFFF03460320FCF7C1
:1045A000EBFF43EA0020D0650620FCF7E5FF034659
:1045B0000420FCF7E1FF43EA002010660720FCF727
:1045C000DBFF107400BD000012000020F0B5384B76
:1045D0000022384E93F908104FF4004503F1800093
:1045E00000290ADD0A2491FBF4F7D0F834C0BF1D7E
:1045F0004CFA07FC5FEACC7713D0002950DA93F825
:104600002340C76AC4F10A04BC4249DA6FF01304BC
:1046100091FBF4F1406BC1F104010841C00738D0AF
:104620003EE0572942DC35615A7193F829204FF456
:104630007A70012A06D0022A08D0032A1AD0042A46
:1046400020D02DE0597EFEF799FD29E0322905DAC8
:10465000597E4FF4FA70FEF791FD21E04A2905DDFD
:10466000597E4FF4FA60FEF789FD19E0597EFEF796
:1046700085FD15E091FBF4F0C8214843597EFEF713
:104680007DFD0DE001EB81008000597EFEF776FD97
:1046900006E035615A71587E41088C20FEF76EFDA8
:1046A00093F90800BDE8F040FCF726B9F0BD000022
:1046B000000000200008014010B54C3800F01AFD41
:1046C000104A114B00F00EFB00F0D0FCC4B2802168
:1046D0000020FDF7A9FD4FF47A70FEF727FE312187
:1046E0000020FDF7A1FDB9210220FDF79DFD4B2122
:1046F0001020FDF799FD2146BDE810400120FDF78F
:1047000093BD00009A9999999999A93F00B5254BB5
:1047100021F0004287B09A4203DC00221346009247
:104720002BE0214B9A4208D140B94FF00100FBF732
:1047300058FEFEF78AFA07B000BD03DBFEF780FAE9
:1047400007B000BD02AAFDF727FE10F003014FF0ED
:1047500001000DD0012914D002291AD00DF1080C46
:104760009CE80F00FDF7DCFF07B081F0004100BDC1
:104770000DF1080C00909CE80F00FEF7A5F807B0BB
:1047800000BD0DF1080C9CE80F00FDF7C9FF07B054
:1047900000BD0DF1080C00909CE80F00FEF794F8A6
:1047A000E2E70000FB21E93F0000F07F2DE9F04146
:1047B00006460F4600F0BCFD041E0D4618BF012042
:1047C000284320F00040C0F17F6000F1E040C00FBE
:1047D0000ED0301C18BF0120384320F00040C0F13B
:1047E0007F6000F1E040C00F04BF0120FBF7F9FD3E
:1047F00020462946BDE8F08100B5124B184693F8D3
:10480000201090F90800002901D0142818DB002896
:1048100002DAD97F022913D046309E2810D20A49E5
:104820004FF40040086114205871597E4FF44870CD
:10483000FEF7A4FC93F908005DF804EBFCF75CB804
:1048400000BD0000000000200008014000B5124B30
:10485000194693F8202091F90810002A01D0142954
:1048600018DB002902DADA7F022A13D046319E29AA
:1048700010D20A4A4FF40041116114215971597E36
:1048800000F52F70FEF77AFC93F908005DF804EB51
:10489000FCF732B800BD0000000000200008014015
:1048A00030B50546002403E0FCF782FE641CE4B248
:1048B000285D002801D00F2CF6D330BD2DE9F04142
:1048C00005460024DFF83C800F4E4FF4B47704EB2C
:1048D000440000EBC4002844B84201DBA0F5B470EA
:1048E00001F088F8414601F0B1F800F0F1FEFEF762
:1048F000CFFC00F009F946F82400641C202CE6DB0C
:10490000BDE8F0814BFA8E3CA40100202DE9F04176
:1049100005460024DFF83C800F4E4FF4B47704EBDB
:10492000440000EBC4002844B84201DBA0F5B47099
:1049300001F060F8414601F089F800F0C9FEFFF788
:10494000E5FE00F0E1F846F82400641C202CE6DBCC
:10495000BDE8F0814BFA8E3C2001002010B5164BCB
:1049600021F00042012486B09A4203DC0022134663
:1049700000941CE0114B9A4208D140B94FF001005D
:10498000FBF72FFDFEF761F906B010BD03DBFEF764
:1049900057F906B010BD02AAFDF7FEFC00F00100B9
:1049A000A4EB40000DF1080C00909CE80F00FEF70E
:1049B00001F806B010BD0000FB21E93F0000F07FC8
:1049C0002DE9F04107468846404600F081FE134E2F
:1049D00004460D46F07C01F025F80146404600F003
:1049E0000BFF394600F0A0FE00F072FE22462B4677
:1049F000FEF74AFA00220A4B00F090FB00F006FB9B
:104A0000F17F072900D10A305A2800DD5A206FF0C3
:104A10005901884200DA0846BDE8F0810000002014
:104A200000804C4070B50646084600F051FE044632
:104A30000D46304600F04CFE22462B46FEF724FA87
:104A40000022034B00F06AFBBDE8704000F0DEBAC4
:104A500000804C4010B5204800F1DB01827D8A7552
:104A6000027D4A704275027A8A70C27DCA70027EE7
:104A70000A71C37B4B71027B8A71427BCA71427C93
:104A80000A72827E4A7202788A72827BCA720279C4
:104A90000A7382784A73427F8A73827CCA73428E19
:104AA0001238140A4C748A7400F18004002B226AB4
:104AB00010D0A262A28C130ACB740A75228D130A3D
:104AC0004B768A7690F822204A75427DCA75C07E60
:104AD000087610BD6262EDE712000020094901F17D
:104AE000E500CA7B42708A7B8270B1F85C20130AB1
:104AF000C3704271B1F86020130A03718271097C9E
:104B0000C17170470000002021F00042A2F1605204
:104B1000B2F5801F01F0004328BFD2F17F6C0BD9A2
:104B20005FEA001C43EAC20242EB507018BF7047B4
:104B300028BF20F001007047B2F5801FBCBF1846A7
:104B400070474FEA410C1CF5001F02D2084601F0E5
:104B500044B870B500F08CFB00000089FFF7F6BF89
:104B60004FF00040A0F580007047000010B591EABA
:104B7000030F48BF83F0004300F1C884841A71EB2F
:104B8000030C05D2121943EB0C03001B61EB0C0163
:104B9000DFF824E14FEA1154A4EB135C1EEA430F43
:104BA00018BF9EEA445F73D023EA0E03DCF1200EA7
:104BB00021EA045143F4801332D322FA0CFE10EBA5
:104BC0000E0023FA0CFE41EB0E01CCF1200E03FA8D
:104BD0000EFE10EB0E0051F10001B1F5801FCCF17B
:104BE000200E32D201EB045112FA0EF2BDE8104051
:104BF00058BF7047401C38BF5FEA420218BF704779
:104C0000002814BF20F0010041F100014FEA4103E8
:104C100013F5001F38BF7047A1F1C04100F076BB0B
:104C2000012A43EB0302ACF1200CDCF11F0E32BF72
:104C30004FF0000E23FA0CF310EB030041EB04518C
:104C4000B4EB115FD0D0A1EB045101F580114908FC
:104C50005FEA300001EB04510ED350F1000038BF81
:104C600012FA0EFE08D1BDE81040C9E7401C38BF5B
:104C70005FEA4202CAD1C3E7BDE810404FEA4103F0
:104C800013F5001F38BF7047A1F1C04100F03EBBD3
:104C90009EEA445F08D011EA5E0FBDE8104004BFF1
:104CA00001F0004100207047BDE8104070B500F0F1
:104CB000DFFA00BF64FBBE3E0000E0FF02494FF098
:104CC000000001F004B800BF0000F87F491058BF91
:104CD000C1F140415B1058BFC3F140438B42EFF339
:104CE000008070472DE9C04130B4DFF8A0C23CEA33
:104CF000111418BF3CEA131400F0EC8081EA03059C
:104D00001CEA111444EAD57418BF1CEA131500F00C
:104D1000C780A4EB05044FF0004545EAC12145EAF0
:104D2000C32341EA505143EA525304F17F7499423C
:104D300004F500344FEAC0204FEAC22208BF904277
:104D400000F09C804FEA13650FF24016765D4FEA43
:104D5000134506FB05F7C7F1807706FB07F74FEA17
:104D6000D737A7FB03687642C8F58038A7FB06CE85
:104D700038BFA8F1010807FB08E64FF0000EA6FBBC
:104D8000028CE6FB03CEDCF1000CCEF1004E38BF06
:104D9000AEF1010EA6FB0C584FF000074FF00005D6
:104DA000E6FB0E87A1FB08C6A0FB07CE16EB0E069E
:104DB00045F10005E1FB076515F1E04E7EBFA4F566
:104DC00080345FEA46066D4116F1800745F1000523
:104DD0004FEA17274FEA066647EA0567A6F1DE465F
:104DE000B6F1805F4FEA15251FD9384624F0010C33
:104DF00005EBC471BCF1FE6F01EB0C1102D8F0BCE5
:104E0000BDE8008124425CBF01F5801E9EEAC47F9C
:104E100002D4F0BCBDE80081244238D4F0BCA1F13A
:104E2000C041BDE8004100F071BA4FEAD22242EA27
:104E300043524FEAD323A7FB02864FEAD02040EA31
:104E4000415007FB03661EEA0E0F4FEAD12105FB16
:104E5000026658BFA6EB0056B6EB00564FEA520E5C
:104E60004EEAC37E18EB0E0E56EB530EBDD518EB73
:104E700002085E417F1C55F10005B6E74FF480152E
:104E80004FF000074FF000064FF00008ADE7F0BC10
:104E90004FF0000001F1C04101F00041BDE8008188
:104EA00011EA0C1F0CEA131500D00CE013EA0C1FDA
:104EB00000F025804FF00000F0BC81EA030101F012
:104EC0000041BDE80081F0BCBDE8004181EA03017A
:104ED00000F01CBAF0BCBDE8004170B500F0C8F9A4
:104EE000097EFC3E00F007B881EA03014FF00000A4
:104EF00001F00041704781EA030100F007BAF0BCFD
:104F0000BDE800414FF0000021497047FFFDFBF96B
:104F1000F7F5F4F2F0EEEDEBE9E8E6E4E3E1E0DEEC
:104F2000DDDBDAD8D7D5D4D3D1D0CFCDCCCBCAC85E
:104F3000C7C6C5C4C2C1C0BFBEBDBCBBBAB9B8B785
:104F4000B6B5B4B3B2B1B0AFAEADACABAAA9A8A878
:104F5000A7A6A5A4A3A3A2A1A09F9F9E9D9C9C9B46
:104F60009A999998979796959594939392919190F1
:104F70008F8F8E8E8D8C8C8B8B8A89898888878782
:104F80008685858484838382828181800000FF07F7
:104F90000000F87F51EA030C17D41CF5801F58BF9E
:104FA000BCF5801F00F10680994218BF704708BF0A
:104FB0009042704707D711F5801F58BF13F5801F27
:104FC00019D499427047894270471CF5801F08D553
:104FD000BCF5801FF7D58B4218BF704708BF8242CF
:104FE00070474FF4001C1CEB410F38BF1CEB430F04
:104FF00001D28B42704770B500F03AF99224490013
:105000004FF000514FF08053FFF760BE4FEA41036D
:105010004FEA5353A3F58063D3F11E03C8BFD3F106
:10502000210C0CDD4FF0004242EAC12242EA50520C
:1050300032FA03FC8CEAE17CACEBE1707047102B98
:10504000C4BF0020704703F5787CBCF1FF3F04D05B
:105050006FF0004282EA2100704770B500F008F955
:105060004992248000207047F2E700004FEA115374
:10507000A3F58063D3F11E03A8BFD3F1200C08DB96
:105080004FF0004242EAC12252EA505232FA03F093
:10509000704709420BD4102BC4BF0020704703F5A2
:1050A000787CBCF1FF3F05D04FF0FF3070474FF0E8
:1050B0000000704770B500F0DBF800BF4992248013
:1050C00000207047F0E710F0004248BF4042B0FABD
:1050D00080F310FA03F10AD0C3F11D0303F58063D6
:1050E0004FEA415002EB035202EBD12170474FF0DF
:1050F00000007047B0FA80F310FA03F10AD0C3F150
:105100001D0303F580634FEA41504FEA035202EB5F
:10511000D12170474FF0000070470000DFF848C110
:1051200070B51CEA111E1EBF1CEA13159EEA0C0F77
:1051300095EA0C0F00F06F8081EA030423EA4C1318
:105140004EEAD47E21EA4C1141F4801143F48013DD
:10515000AE44A1FB024CA0FB0365AEF17F7E361985
:1051600055EB0C05A1FB034C4CF10003A0FB021C0A
:1051700016EB0C06654153F10003094218BF46F0D7
:10518000010613F4007F0BD14FEA03314FEA0530DB
:10519000340341EA155140EA16506FF003020AE069
:1051A0004FEAC3214FEAC520F40241EA555140EAD3
:1051B00056506FF0020202EB2E4201EB025585EAD7
:1051C000CE710AD05FEA440C18BF24F0004450F1BD
:1051D000000041F1000120EAD47040F2FE7C6245FB
:1051E00000D270BDA84214BF4FF080444FF040443D
:1051F000002E08BF0024BEF1806FA8BFA1F1C041FE
:10520000BDE8704080F282804FF0000001F1C041A3
:1052100001F0004170479EEA0C0F0CEA131518BF0D
:1052200095EA0C0F06D04FF0000081EA030E0EF055
:10523000004170BD00F01CF88900013E00F007B885
:1052400000F009B84FEA430C5FEA5C5C08D081EAE1
:10525000030100F05BB84FEA410C5FEA5C5CF6D1F9
:105260004FF00000014970470000FF070000F87F81
:105270000EF1020E2EF0030E5EF8046B364205D4DA
:10528000012A43EB030515F5001F12D8012841EB55
:10529000010C1CF5001F0CD80ED14FEAD17C15F57E
:1052A000001F0CEB4C0C0CF1020C08BF4CEBD37C38
:1052B00004E04FF0080C01E04FEAD37C0CEB4C0506
:1052C00026FA05F606F00706B6F1040C06D20EEB38
:1052D000860CBDE870404CF0010C6047DFE80CF034
:1052E000090B02024FF000414FF00000A1F5002130
:1052F00070BD19461046012851EB010418BFD4F5C2
:10530000001484BF002001F0004170BD0808A0F522
:1053100000114FEA3101704791EA030F10B581F097
:1053200000413FF52BAC83F0004300F0EFB80000E4
:105330002DE9F04101F5801CBCF5001FC0F2C380CF
:105340004FEA115C21EA0C510CF1FD0C41F4801183
:105350005FEA5C0C0CF5C07C01D3400049413DA4E0
:10536000890241EA905187028E0E0A0CA45D04FB6B
:1053700004F602FB06F6C6F14046A4FB0662F60DF3
:1053800046EA422606FB06F4A4FB01235242C3F17F
:10539000404338BF5B1EA6FB02420024E6FB032409
:1053A000D20B42EA4446A6FB0623A1FB02E2A3FB82
:1053B00007E4A4184FF0000252F10002E3FB01429F
:1053C0006442C2F1404E38BFAEF1010EA6FB042389
:1053D0004FF00002E6FB0E32A2FB03464FF0000442
:1053E000B61954F10004E2FB0264A1FB06E6A4FB3B
:1053F00007E816EB08064FF0000858F10008E4FB38
:1054000001687642C8F1405838BFA8F10108A2FBF4
:1054100006E4A3FB08E52D194FF0000454F1000445
:10542000E2FB0854A1FB05E6A7FB04E818EB06081D
:105430004FF0000656F10006E1FB048618F1200546
:1054400056F10006A809A8F11B08B10908F03F08A9
:10545000B8F10A0F40EA86601CD901EB0C51BDE897
:10546000F08100BFFCF5EEE8E2DDD8D3CFCBC7C3B7
:10547000C0BDB9B6B4B1AEACA9A7A5A3A19F9D9B71
:105480009A9896959392908F8D8C8B898887868534
:1054900084838281A0FB006800FB01F208EB4208D4
:1054A000B8EB872807D5341858EB0104D5D5401C34
:1054B00051F10001D1E7341A78EB0104CDD4401E3C
:1054C00071F10001C9E75FEA4C0C5FEA9C5C0DD109
:1054D00005D34FF0000001F00041BDE8F081BDE8C8
:1054E000F04170B5FFF7C4FE6DDBFFBEBDE8F041D3
:1054F0004FF00000004970470000F87F10B591EAB6
:10550000030F48BF83F000433FF538AB841A71EBBB
:10551000030C07D212198CF0004C43EB0C03001B58
:1055200061EB0C01DFF8A4E14FEA1154A4EB135C2A
:105530001EEA430F18BF9EEA445F00F0B08023EAE2
:105540006E03524221EA0451C3EB6E0338BF5B1E67
:10555000DCF1200E25D322FA0CFE10EB0E0043FAEC
:105560000CFE41EB0E01CCF1200E03FA0EFE10EB07
:105570000E0051F10001CCF1200E29D412FA0EF2E6
:1055800001EB0451BDE8104058BF7047401C1CBFE0
:10559000B2F1004F704700280CBF491C20F00100F9
:1055A000704712EB020E43EB030218BF4FF0010EDF
:1055B0004EEA4202ACF1200CDCF11E0E54D943FA43
:1055C0000CFE10EB0E0051F1FF31CCF11E0ED5D5C3
:1055D0000EF1010E12FA0EFE404141EB010101EB0A
:1055E000445C5FEA5C5C10D910EBDE7001EB0451A7
:1055F00038BFBEF1004FBDE8104018BF704700280B
:105600000CBF491C20F00100704730D24FEAD42C67
:1056100011F5001124F400641BD0B1FA81F20B3AA9
:10562000A41AA41ED2F12003914030FA03F31943C7
:10563000904001EBCC71002C01EB0451BDE810400F
:10564000A8BF704701F1C0414FF0000001F00041D8
:105650007047B0FA80F310FA03F100D110BDE41ADC
:10566000173C4805C90AE4E701EB045110BD491095
:1056700001EB0451BDE810404FEA300002E04FF06A
:10568000000170474A0008BF0042F8D0B2F5001F81
:1056900028BF704701F000414FF0000070479EEABC
:1056A000445F07D011EA5E0FBDE8104004BF00213F
:1056B00000207047BDE8104070B5FFF7D9FD00BF6E
:1056C00040DFF63E83F00041104670470000E0FFE7
:1056D00043004FEAD30C4FEA3C0C43401FBF400746
:1056E0000CF1605113F0FE4F70471CF0006F03D1B6
:1056F00000200CF0004170470CF0004343EA50706A
:1057000010B540EACC0000F022FA00BF0000009281
:105710004FEA0001FFF7FABD4FF000414FF00000E3
:10572000A1F500217047000090EA010F48BF81F009
:10573000004100F15E82421A3CBF801A89184FEA8C
:10574000D0524FF07F4C1CEA410FA2EBD15318BF4F
:105750009CEA026F00F03B804FF0004C4CEA0020C6
:105760004CEA012121FA03FC10EB0C0C1ED202F1D1
:10577000FF325FEA1C2040EBC25038BF70471CF07C
:105780007F0F4FEA400C18BFBCF17F4F38BF704706
:10579000C3F12003994008BF20F00100BCF17F4F06
:1057A00038BF7047A0F1C04000F017BA4FEA3C0084
:1057B000000A40EBC25028BF1CF0FF0F4FEA400C1C
:1057C000E6D018BFBCF17F4F38BF7047EAE79CEACC
:1057D000026F05D010EA5C0F08BF00F00040704770
:1057E00010B500F0B4F900BF64FBBE3E014800F004
:1057F0006EBA00BF0000C07F4FF47F0C1CEAD012CD
:105800001EBF1CEAD11392EA0C0F93EA0C0F00F0B2
:10581000858090EA010F48BF42F4807240F4000C8A
:1058200041F400002CF07F4120F07F4000B5814220
:10583000A2EB03020FF2081CACEB504EC0F10000CB
:105840009EF800E04FEA4E0E00FB0EFC38BF490008
:105850004FEA2C1C02F5FA020CFB0EF34FEACE1EA7
:105860004FEA112C4FEAC1210EEB635E42EB22425C
:105870000EFB0CFC4FEA1C5300FB03114FEA112CEA
:105880004FEA01310EFB0CFC4FEADC4C00FB0C1123
:10589000C14228BF09184CEB03335DF804EB10EB51
:1058A000410143EBC250B2F57C0F38BF704729D598
:1058B00012F0F00F1CBF00F1C04000F00040704734
:1058C000008182838485868788898B8C8D8E8F91D9
:1058D0009293959697999A9C9D9FA0A2A3A5A7A8FD
:1058E000AAACAEB0B2B3B5B7B9BCBEC0C2C5C7C929
:1058F000CCCED1D4D7D9DCDFE2E6E9ECF0F3F7FA8D
:10590000FE0000004FEA400C0CF1807CBCF17E4FA1
:1059100028BF7047B0F1C04000F05FB990EA010FB6
:105920000CEAD11348BF42F48072624538BF634528
:1059300007D213F47F0F16D080EA010000F0004078
:10594000704710B500F003F9097EFC3E00F005B881
:1059500080EA010000F00040704780EA010000F09A
:10596000004000F03AB912F47F0F04BF02487047BC
:1059700080EA010000F031B90000C07F41000B0E49
:10598000D3F19E0208D950F400034FEA032323FA0F
:1059900002F048BF4042704710B500F0D8F800BF91
:1059A00049922480002070476FF0004282EA200074
:1059B00070470000C10DD1F19E0206DB4FEA0023C3
:1059C00043F0004323FA02F07047004207D54FEA44
:1059D0004001B1F1FE4F02D24FF00000704710B508
:1059E00000F0B5F849922480002070476FEA20004B
:1059F0007047000010F0004148BF4042B0FA80F309
:105A000010FA03F2C3F19D030BD051EAC35101EB2D
:105A10001220530638BF704700F1010008BF20F084
:105A200001007047B0FA80F310FA03F2C3F19D034E
:105A30000AD0D90501EB1220530638BF704700F198
:105A4000010008BF20F00100704700004FF47F0CF8
:105A50001CEAD0121EBF1CEAD11392EA0C0F93EA83
:105A60000C0F00F0478090EA010F48BF42F48072AB
:105A70004FF0004C4CEA00204CEA012102EB0302FB
:105A8000A0FB0113A2F50002002918BF43F0010397
:105A90005B0028BF4FEA330342EB22425FEA132C3C
:105AA0004CEBC2502EBFBCEB436FB2F57C0F70477E
:105AB0004FEA036CBCF1004F08BF20F00100B2F5C3
:105AC0007C0F38BF70470BD582F0FF0212F5803F84
:105AD000C8BF704700F1C040D8BF00F00040704719
:105AE00000F5000C5FEA4C0C48BF7047B0F1C040B5
:105AF00000F073B890EA010F0CEAD11348BF42F4EA
:105B00008072624538BF634504D280EA010000F02C
:105B10000040704710B500F01AF800BF8900013E40
:105B200000F007B800F009B85FEA410C5FEA1C6CAE
:105B300008D080EA010000F050B85FEA400C5FEA4C
:105B40001C6CF6D14FF00040A0F5800070470EF1BC
:105B5000020E2EF0030E5EF8044B244204D44FEAEA
:105B60004102B2F17F4F11D84FEA4003B3F17F4FAA
:105B70000CD80ED14FEAD07CB2F17F4F0CEB4C0C1D
:105B80000CF1020C08BF4CEBD17C04E04FF0080C88
:105B900001E04FEAD17C0CEB4C0324FA03F404F04F
:105BA0000704B4F1040C06D20EEB840CBDE81040DF
:105BB0004CF0010C6047DFE80CF0070802024FF0E0
:105BC0000040A0F5800010BD0846420018BFD2F189
:105BD000807288BF00F0004010BDFF2141EAD05024
:105BE000C005704790EA010F48BF81F000413FF5C2
:105BF000A2AD421A04D882F00042A0EB0200114488
:105C00004FEAD0524FF07F4C1CEA410FA2EBD15328
:105C100018BF9CEA026F4AD04FF0004C4CEA0020BB
:105C20004CEA012121FA03FCB0EB0C0C0FD412F06A
:105C3000FE0F36D05FEA4C001DD5001240EBC2507B
:105C400038BF70471CF03F0F18BF70470BE0A2F140
:105C500001025FEA1C2040EBC25038BF70471CF0C5
:105C60007F0F18BF7047C3F12003994014BF401E37
:105C700020F00100704780084FEA122308BF7047E8
:105C8000B0FA80FCA2EB0C02CCF1280C60FA0CF00C
:105C900093EA122F04BF00EBC25070474FEAC37063
:105CA0007047130A5FEADC1008BF7047F6E79CEA0A
:105CB000026F04D010EA5C0F08BF0020704710B5D7
:105CC000FFF745FF40DFF63E81F0004070470CF0E3
:105CD0000F03092B08BF082000F07F800A2B0BD090
:105CE000082B18BF704708BF1CF0400F0AD04FF0B8
:105CF00000004FF0000170471CF0400F18BF4FF03C
:105D0000004070471CF0100F08D020F0704300F0E6
:105D10007F4242EAD3014FEA4370704700F060408F
:105D200021F07F4242EA000201F07F4040EA7270B7
:105D300070474FF0FF0C4CF4E06C1CEA11531CBF91
:105D40009CEA030C9445C2BFDA4201EB0251704752
:105D5000002B0DD0BCF1000F0FD0002A01F0004144
:105D6000A4BF41F0E04141F07F614FF00000704777
:105D700001F000414FF00000704750EA01334FF04E
:105D80009B0C18BF4CF0806C7EF498AF70474FF0BE
:105D9000FF0212EAD0521CBF92F0FF038B42C2BF37
:105DA000D14200EBC1507047002A0AD0002B0BD023
:105DB000002900F00040A4BF40F0FE4040F4000085
:105DC000704700F00040704743024FF00B0C18BFC3
:105DD0004CF0806C7FF40AAD70471CF4801F11D02A
:105DE0001CF4E02F03D06FEACC31490070474FF02C
:105DF0004050EFF3008222F0704242EA000282F348
:105E0000008870474FF00000704700000000040455
:105E1000040000080000000800000000000000006E
:105E20000102030406070809000000000102030440
:105E300067A029BD9C5775BD6FD1A5BD4AC9D4BD0A
:105E4000F8C102BEE1D3533FF8C102BE4AC9D4BD76
:105E50006FD1A5BD9C5775BD67A029BD84B46FBD2A
:105E60005893B5BDDB14FCBD17B123BE66BE5D3FC4
:105E700017B123BEDB14FCBD5893B5BD84B46FBD10
:105E800014BEA1BD6FEDFCBDDC252FBEE9383F3F40
:105E9000DC252FBE6FEDFCBD14BEA1BD5BC0FF3C79
:105EA00045D0BF3D45D0BF3D5BC0FF3C0000803FBB
:105EB000D417A5BFF8782A3FE66401BED315003F8A
:105EC000D315003F00000000000000000000803FEC
:105ED000589B2E3A00000000000000000000000067
:105EE00004FA97999999D93FAF788E1DC571CC3F27
:105EF0009FC678D0099AC33F935555555555E53FF0
:105F0000599322942449D23FDE03CB966446C73F7F
:105F100044523EDF12F1C23F4FBB610567ACDD3F2B
:105F2000182D4454FB21E93F9BF681D20B73EF3FC0
:105F3000182D4454FB21F93FE2652F227F2B7A3C38
:105F4000075C143326A6813CBDCBF07A8807703CF1
:105F5000075C143326A6913CC4EB98999999C9BF64
:105F6000711623FEC671BCBF6D9A74AFF2B0B3BF99
:105F70009AFDDE522DDEADBF2F6C6A2C44B4A2BF59
:105F80000D5555555555D53FFF8300922449C23FC5
:105F90006E204CC5CD45B73F513DD0A0660DB13FF9
:105FA000EB0D76244B7BA93F11DA22E33AAD903F0B
:105FB0004C5555555555A53F7751C1166CC156BF27
:105FC0009015CB19A001FA3EAD529C804F7E92BE37
:105FD000C4B1B4BD9EEE213ED43888BEE9FAA8BD56
:105FE000000000000000000000004054FB21F93FC9
:105FF0003163621A61B4D03D0000601A61B4D03DD3
:106000007370032E8A19A33B0000002E8A19A33B4C
:10601000C14920259A837B39000000000000000060
:106020006E83F9A22915444ED15727FCC0DD34F503
:10603000999562DB4190433CAB6351FE61C5BBDE89
:106040003A6E24B7E0D24D42EA2E49061C92D1099D
:106050001CEB1DFE3EA729B1F53582E88444BB2E1A
:1060600026709CE9417E5FB439D69139F439538367
:106070008B5F849C3B28F9BDFF97F81F0F9805DEC6
:106080008B112FEF1F6D0A5ACF7E366DB709CB27C4
:10609000663F464F2DEA5F9EC7BA27757BF1E5EB59
:1060A000F739073DEA92528AB15FFB6B085D8D1F9D
:1060B000A6F810111111813FD561C119A0012ABFA5
:1060C0007DFEB157E31DC73EEB9C2B8AE6E55ABE29
:1060D0007CD5CF5A3AD9E53D7AFE10111111C13F56
:1060E00037D60684F464963F280356C9226D6D3F67
:1060F0000165F2F2D844433FA69237A0887E143F50
:10610000735360DBCB75F3BEFE41B31BBAA1AB3F4B
:1061100093846EE9E326823F1583E0FEC8DB573F98
:1061200068108D1AF726303FE9A7F0320FB8123FFA
:10613000D47ABF74702AFB3E58610008000000202A
:1061400020010000280100087862000820010020DA
:10615000500F000044010008000000000000010092
:10616000000000000000000000000000000000002F
:10617000000000000000000000000000000000001F
:10618000000000000000000000000000000000000F
:10619000475167F7000000000AD723BD0000000048
:1061A00000000000000000000000000000000000EF
:1061B00000000000000000000000000000000000DF
:1061C00000000000000000000000000000000000CF
:1061D00000000000000000000000000000000000BF
:1061E00000000000000000000000000000000000AF
:1061F000000000000000000000000000000000009F
:10620000000000000000000000000000000000008E
:10621000000000000000000000000000000000007E
:10622000000000000000000000000000000000006E
:10623000000000000000000000000000001300004B
:106240000000000000000A010202010801070158D5
:1062500000005D002C0100F900BE0F010100B40038
:10626000000000000000000001000000100000001D
:08627000000000000024F4000E
:04000005080000ED02
:00000001FF
